:100000000B2CFF3FFF3FFF3F70082000A40071084A
:10001000A3007208A2007308A10080310B1D1428F0
:10002000B80A0319B90A0B11911E6E2823009D18F6
:100030001B2873101C2873141D1920280310212855
:1000400003147318272803182728731028287314FB
:10005000731C3728230019082000B10023009D13CA
:100060002000AB0A0319AC0A23009D1716282300B1
:1000700019082000B10031080D3A0130031D00308D
:10008000F1008030F00080302E067002031D4A28F7
:100090002D081F3C013003180030F0007108F004F7
:1000A0000319602820302D07860001302E3D87007F
:1000B00081010130C6000030C700210091126C2878
:1000C000203020002D07860001302E3D87003108AA
:1000D0008100AD0A0319AE0A20009112111CA1285B
:1000E0000B309700DB309600AF0A0319B00A3008D6
:1000F000003C031D7D282F08073C0318A028150885
:10010000C200C3013808F100F0017008BE07710891
:10011000BF3D0030C03DC13D4208BE074308BF3D62
:100120000030C03DC13D9501B801B9011030220039
:100130008C062000AF01B0010130A9000030AA00F8
:1001400011102408F0002308F1002208F200210811
:10015000F300090023009E18AF280000AA28200001
:100160006B0823009A00080071088A00700882005A
:1001700008002000F801F9011030FC00710DF80DA5
:10018000F90D7408F8027508031C750FF9020318BD
:10019000D0287408F80775080318750FF9070310BD
:1001A000F00DF10DFC0BBE2808002000FB01FA0148
:1001B000F901F801A001730DF80D7408F802750833
:1001C000031C750FF9027608031C760FFA027708F4
:1001D000031C770FFB020001031C0130A002F30D8A
:1001E0000730FC00730DF80DF90DFA0DFB0DA00D95
:1001F0007408731C0D29F8027508031C750FF902A9
:100200007608031C760FFA027708031C770FFB02AF
:100210000001031C0130A0021E29F807750803180D
:10022000750FF90776080318760FFA077708031891
:10023000770FFB07000103180130A007F30DFC0B3B
:10024000F228720DF80DF90DFA0DFB0DA00D7408D2
:10025000731C3C29F8027508031C750FF902760817
:10026000031C760FFA027708031C770FFB020001CC
:10027000031C0130A0024D29F80775080318750FFB
:10028000F90776080318760FFA0777080318770F2F
:10029000FB07000103180130A007F20D0730FC0036
:1002A000720DF80DF90DFA0DFB0DA00D7408721CFE
:1002B0006B29F8027508031C750FF9027608031CF8
:1002C000760FFA027708031C770FFB020001031C6C
:1002D0000130A0027C29F80775080318750FF9078B
:1002E00076080318760FFA0777080318770FFB07CD
:1002F000000103180130A007F20DFC0B5029710D0D
:10030000F80DF90DFA0DFB0DA00D7408721C9A2959
:10031000F8027508031C750FF9027608031C760FA6
:10032000FA027708031C770FFB020001031C01305F
:10033000A002AB29F80775080318750FF9077608AE
:100340000318760FFA0777080318770FFB070001E9
:1003500003180130A007F10D0730FC00710DF80DF6
:10036000F90DFA0DFB0DA00D7408711CC929F802D6
:100370007508031C750FF9027608031C760FFA0244
:100380007708031C770FFB020001031C0130A00259
:10039000DA29F80775080318750FF90776080318A6
:1003A000760FFA0777080318770FFB070001031889
:1003B0000130A007F10DFC0BAE29700DF80DF90D01
:1003C000FA0DFB0DA00D7408711CF829F8027508D0
:1003D000031C750FF9027608031C760FFA027708E2
:1003E000031C770FFB020001031C0130A002092A45
:1003F000F80775080318750FF90776080318760FC4
:10040000FA0777080318770FFB070001031801307C
:10041000A007F00D0730FC00700DF80DF90DFA0D76
:10042000FB0DA00D7408701C272AF8027508031C28
:10043000750FF9027608031C760FFA027708031C81
:10044000770FFB020001031C0130A002382AF807D5
:1004500075080318750FF90776080318760FFA0761
:1004600077080318770FFB07000103180130A00776
:10047000F00DFC0B0C2A70184B2A7408F80775084D
:100480000318750FF90776080318760FFA0777082F
:100490000318770FFB0708002000520886006A083F
:1004A0008100860A5008F0005108F100B4200800CD
:1004B0002000E30160088400610885000008E20074
:1004C0006208003A0319722A6208EB00AA20200091
:1004D000E30A6308600784000030613D850000087E
:1004E000E200602A0800200062088400630885009A
:1004F0000008F00070080319902A6208840063085D
:1005000085000008F0006008860061088700700818
:100510008100E00A0319E10AE20A0319E30A732AD7
:10052000600886006108870081010800AA30200069
:10053000D0000030D1006B30D2000030D300FF304B
:10054000CC00FF30CD000030CE000030CF00FF30B7
:10055000D400FF30D5000030D6000030D700FF3087
:10056000D800FF30D9000030DA000030DB00230073
:100570009E1690309D0021008C140C142000911EBA
:10058000C52A23001908F000BE2A08002200A00195
:100590002000CA01CB01AD01AE01C601C701F101C6
:1005A000F20180307206F00080307002031DDA2AFA
:1005B000203071020318E72A2030710786000130CD
:1005C000723D87008101F10A0319F20AD12A230042
:1005D0001908F100F20121009116080012001E0016
:1005E000F003031DEE2AF103031DEE2A080020008C
:1005F00060088400610885000008F0007008031995
:100600000D2B60088400610885000008EB00AA201B
:100610002000E00A0319E10AF72A0800200011105F
:100620000B309700DB30960099019912A901AA01BD
:10063000313098002100111008002100151195108B
:100640001510951595160B118B12200095019E0122
:1006500008002000E401053064020318392B640807
:10066000620786000030633D870020308100E40A85
:100670002B2B6408620786000030633D87008101F0
:10068000E40364086207E5000030633DE6000A30D9
:10069000F400F5016008F0006108F100B920780865
:1006A000F0007908F1003030F00765088600660830
:1006B0008700700881000A30F400F5016008F0003E
:1006C0006108F100B9207008E0007108E100003015
:1006D0007106031D6D2B00307006031D702B722BED
:1006E000E403412B08000D302000EA004C220A30C0
:1006F0002000EA004C2208002000E301600884008A
:10070000610885000008E2006208003A0319962B90
:100710006208EA004C222000E30A630860078400B4
:100720000030613D85000008E200842B08002000B5
:10073000E601E70100306702031DA02B0A306602C4
:100740000318AE2B6608640786006708653D8700BE
:1007500020308100E60A0319E70A9A2B660864072D
:1007600086006708653D870081010130E6020030A0
:10077000E73B66086407E8006708653DE9000A3062
:10078000F400F501F601F7016008F0006108F100DE
:100790006208F2006308F300D5207808F0007908B9
:1007A000F1007A08F2007B08F3003030F0076808A7
:1007B000860069088700700881000A30F400F5019E
:1007C000F601F7016008F0006108F1006208F2002C
:1007D0006308F300D5207008E0007108E10072089A
:1007E000E2007308E3000030F4007306031D022CDE
:1007F00074087206031D022C74087106031D022C76
:100800007008003A031D052C0A2C0130E602003066
:10081000E73BB92B080007302000A500A601A7017F
:10082000A8017830210099000B30FB002630FC0035
:100830005D30FD00FD0B1A2CFC0B1A2CFB0B1A2C47
:100840000000000023008C01033024008C002200F3
:10085000910192012500930122009D019D149D1399
:100860001D11063021008C008B01200091019201A6
:100870000B138B130730A500A601A701A801C62200
:10088000A0302000B6000030B70023009F15CF3005
:100890009B009C011E1596220B30FB002630FC00AD
:1008A0005D30FD00FD0B522CFC0B522CFB0B522C2F
:1008B00000000000063021008C002000BE01BF01B6
:1008C000C001C101C201C301B801B901BA01BB0134
:1008D000BC01BD01C401C501C801C901CA01CB01E8
:1008E0000C30EA004C220B30FB002630FC005D305F
:1008F000FD00FD0B792CFC0B792CFB0B792C0000F7
:1009000000002000C601C701AD01AE017323200025
:100910003608E0003708E1001430E2008730E300D9
:100920007322A030B6000030B7003608E000370868
:10093000E10058223608E0003708E1003930E200D3
:100940008730E3007322A030B6000030B7003608CD
:10095000E0003708E10058223608E0003708E100DF
:100960005630E2008730E3007322A030B60000303A
:10097000B7003608E0003708E10058227323A030A2
:100980002000B6000030B700AF01B001AB01AC01F0
:10099000B10123009D011D169D179D161908200009
:1009A000B100EF30E0008630E100F7227323200031
:1009B000B401B501B201B3011D2395010E238B16BD
:1009C0000B112000181411102100911611140B178F
:1009D0008B172000BE01BF01C001C101C201C301CC
:1009E000B801B901BA01BB01BC01BD01CA01CB010B
:1009F000C401C501C801C901CA0A0319CB0A0030E4
:100A00004706031D052D01304606031D1D2D5230DE
:100A1000EA004C223D302000EA004C222030200029
:100A2000E0000130E1007C23C601C701B101AD0146
:100A3000AE01AB01AC0121009116003020002A0666
:100A4000031D242D00302906031D2B2D3808DE0040
:100A50003908DF001D2DA901AA014308003C031D30
:100A6000332D4208003C0318DD2DA030B6000030C5
:100A7000B7004A08E0004B08E1003608E2003708FA
:100A8000E30029233608E0003708E1007C23093021
:100A9000EA004C22A0302000B6000030B7009C30A5
:100AA000E0008730E100F7224208E0004308E1005F
:100AB0003608E2003708E30029233608E00037084B
:100AC000E1007C230930EA004C2220003608E000D7
:100AD0003708E1007C230930EA004C22B1302000C5
:100AE000E0008730E100F722A030B6000030B70008
:100AF0003E08E0003F08E1004008E2004108E30052
:100B00003608E4003708E50097233608E000370888
:100B1000E1007C230930EA004C22BB302000E000D9
:100B20008730E100F7227D30F400F501F601F7018E
:100B30003E08F0003F08F1004008F2004108F300D1
:100B4000D5207008BA007108BB007208BC00730899
:100B5000BD007008E0007108E1007208E20073084F
:100B6000E3003608E4003708E50097233608E00084
:100B70003708E1007C23C230E0008730E100F72233
:100B8000A030B6000030B7004408E0004508E1009E
:100B90003608E2003708E30029233608E00037086A
:100BA000E1007C230930EA004C2273232000C40AB0
:100BB0000319C50AC801C901452EC80A0319C90A83
:100BC0003C30F4000030F5004A08F0004B08F1001A
:100BD000B9207808F0007908F10000307106031D93
:100BE000F32D00307006031D452EA030B6000030F6
:100BF000B7004A08E0004B08E1003608E200370879
:100C0000E30029233608E0003708E1007C2309309F
:100C1000EA004C22A7302000E0008730E100F722F4
:100C2000A030B6000030B7003E08E0003F08E10009
:100C30004008E2004108E3003608E4003708E50018
:100C400097233608E0003708E1007C230930EA00EA
:100C50004C22C7302000E0008730E100F722A030AE
:100C6000B6000030B7004808E0004908E100360847
:100C7000E2003708E30029233608E0003708E100E6
:100C80007C230930EA004C227323200045080B3CEA
:100C9000031D4C2E4408B83C0318CD2E7130E000E3
:100CA0008730E100F722DC01DD0101305D02031D28
:100CB0005B2E2C305C0203186E2E203022008C0636
:100CC0001030FC009430FD00FD0B642EFC0B642EF4
:100CD00000002000DC0A0319DD0A552E0530FB0058
:100CE0000F30FC00F130FD00FD0B742EFC0B742E58
:100CF000FB0B742EDC01DD0101305D02031D822E31
:100D00002C305C020318952E203022008C06063011
:100D1000FC003030FD00FD0B8B2EFC0B8B2E0000F9
:100D20002000DC0A0319DD0A7C2E0530FB000F30A1
:100D3000FC00F130FD00FD0B9B2EFC0B9B2EFB0BF2
:100D40009B2EDC01DD0101305D02031DA92EF43074
:100D50005C020318BC2E203022008C060B30FC00F5
:100D60006230FD00FD0BB22EFC0BB22E0000200005
:100D7000DC0A0319DD0AA32E0230FA003130FB0031
:100D80006230FC004530FD00FD0BC42EFC0BC42E70
:100D9000FB0BC42EFA0BC42E4E2E4908013C031D3A
:100DA000D32E48082C3C0318ED2E8930E000873004
:100DB000E100F72273232000CA01CB01C401C50161
:100DC0009501B801B901BE01BF01C001C101BA015D
:100DD000BB01BC01BD01C801C901FC2CEE2E493488
:100DE0005434203455344134523454342034523441
:100DF000413430342D3452344134313420342634AB
:100E00002034543469346D346534723430342034D1
:100E100026342034543469346D34653472343134BA
:100E200020340A340D34003446346C346F34773453
:100E30006D34653474346534723420346F346E34F8
:100E40002034433475346C346C3469346734613421
:100E50006E34203457346134743465347234203441
:100E60004F34753474346C34653474340D340A344E
:100E7000003431343234463431343834343430345C
:100E8000203420346134763465346334203469345A
:100E90006E3474346534723466346134633465346A
:100EA0002034323454340D340A340034323437347C
:100EB0002F34303438342F343134343420344D34FA
:100EC00069346B3472346F344334203450347234A8
:100ED0006F34203436342E34343430340D340A3404
:100EE00000342034203441344C34413452344D34B5
:100EF0004534203444344534423449345434203465
:100F0000453447344F345534543420340D340A3486
:100F10000034503461347334203464346534203404
:100F20006434653462346934743420342E342E349D
:100F300020344F344B34003420344E346234503437
:100F40002F347334653463343D342034003420341A
:100F500054346F34743461346C3450343D34203440
:100F60000034203454346F34743461346C3450346D
:100F70003D342034003420344E3462344C343D341B
:100F80002034003420344B343D34203400342034B9
:100F90004C343D3420340034FF3FFF3FFF3FFF3FE0
:020000040001F9
:04000E00C4291334BA
:020000040001F9
:10E000004D0065007300750072006500200064001B
:10E010006500200044006500620069007400200073
:10E0200020004500610075002000410064006F0081
:10E03000750063006900730073006500750072006D
:10E04000430075006C006C006900670061006E00A1
:10E0500020000D000A000000FF00FF00FF00FF008D
:10E0600050004900430031003200460031003800C2
:10E070003400300020002B00200049006E007400A6
:10E0800066006100630065002000630061007000AD
:10E0900074006500750072002000640065002000B7
:10E0A0002000640065006200690074000D000A0031
:10E0B0000000FF00FF00FF00FF00FF00FF00FF0067
:10E0C0004D0069006B0072006F004300200050009B
:10E0D00072006F00200036002E0034003000200057
:10E0E000200072006500670069007300740065001D
:10E0F0007200650064000D000A00000000000000CE
:10E10000FF00FF00FF00FF00FF00FF00FF00FF0017
:10E11000FF00FF00FF00FF00FF00FF00FF00FF0007
:10E12000FF00FF00FF00FF00FF00FF00FF00FF00F7
:10E13000FF00FF00FF00FF00FF00FF00FF00FF00E7
:10E1400049006E0069007400200048004300300060
:10E150003600200042006C006500750000000000E1
:10E16000FF00FF00FF00FF00FF00FF00FF00FF00B7
:10E17000FF00FF00FF00FF00FF00FF00FF00FF00A7
:10E18000FF00FF00FF00FF00FF00FF00FF00FF0097
:10E19000FF00FF00FF00FF00FF00FF00FF00FF0087
:10E1A0002A00FF00FF00FF00FF00FF00FF00FF004C
:10E1B000FF00FF00FF00FF00FF00FF00FF00FF0067
:10E1C0007000610075006C0066006A0075006A00EE
:10E1D0006F002E0066007200650065002E0066006C
:10E1E00072000D000A000000FF00FF00FF00FF00AA
:10E1F000FF00FF00FF00FF00FF00FF00FF00FF0027
:00000001FF
